:020000040800F2
:100000000050002025130008C9120008CF12000874
:10001000D5120008DB120008E11200080000000001
:10002000000000000000000000000000E7120008CF
:10003000F312000800000000FF1200080B13000874
:100040006D1300086D1300086D1300086D13000890
:100050006D1300086D1300086D1300086D13000880
:100060006D1300086D1300086D1300086D13000870
:100070006D1300086D1300086D1300086D13000860
:100080006D1300086D1300086D1300086D13000850
:100090006D1300086D1300086D1300086D13000840
:1000A0006D1300086D1300086D1300086D13000830
:1000B0006D1300086D1300086D1300086D13000820
:1000C0006D1300086D1300086D1300086D13000810
:1000D0006D1300086D1300086D1300086D13000800
:1000E0006D1300086D1300086D1300080000000078
:1000F0000000000000000000000000000000000000
:0C01000000000000000000005FF808F1A3
:1001100010B5054C237833B9044B13B10448AFF341
:1001200000800123237010BD140000200000000097
:10013000F032000808B5034B1BB103490348AFF385
:10014000008008BD0000000018000020F032000808
:1001500070B54FF0FF0C4CF4E06C1CEA11541DBF5D
:100160001CEA135594EA0C0F95EA0C0F00F0DEF828
:100170002C4481EA030621EA4C5123EA4C5350EA0D
:10018000013518BF52EA033541F4801143F480135E
:1001900038D0A0FB02CE4FF00005E1FB02E506F0EF
:1001A0000042E0FB03E54FF00006E1FB03569CF044
:1001B000000F18BF4EF0010EA4F1FF04B6F5007F4A
:1001C00064F5407404D25FEA4E0E6D4146EB0606BC
:1001D00042EAC62141EA55514FEAC52040EA5E5045
:1001E0004FEACE2EB4F1FD0C88BFBCF5E06F1ED8EF
:1001F000BEF1004F08BF5FEA500E50F1000041EB26
:10020000045170BD06F0004646EA010140EA0200D2
:1002100081EA0301B4EB5C04C2BFD4EB0C0541EAF4
:10022000045170BD41F480114FF0000E013C00F309
:10023000AB8014F1360FDEBF002001F0004170BD2D
:10024000C4F10004203C35DA0C341BDC04F1140446
:10025000C4F1200500FA05F320FA04F001FA05F2D2
:1002600040EA020001F0004221F0004110EBD3709F
:1002700021FA04F642EB06015EEA430E08BF20EACB
:10028000D37070BDC4F10C04C4F1200500FA04F36E
:1002900020FA05F001FA04F240EA020001F0004100
:1002A00010EBD37041F100015EEA430E08BF20EA73
:1002B000D37070BDC4F1200500FA05F24EEA020EBB
:1002C00020FA04F301FA05F243EA020321FA04F0EA
:1002D00001F0004121FA04F220EA020000EBD370A1
:1002E0005EEA430E08BF20EAD37070BD94F0000FA1
:1002F0000FD101F00046400041EB010111F4801FD5
:1003000008BF013CF7D041EA060195F0000F18BF85
:10031000704703F00046520043EB030313F4801FC1
:1003200008BF013DF7D043EA0603704794EA0C0F7B
:100330000CEA135518BF95EA0C0F0CD050EA410691
:1003400018BF52EA4306D1D181EA030101F000410E
:100350004FF0000070BD50EA410606BF1046194636
:1003600052EA430619D094EA0C0F02D150EA013642
:1003700013D195EA0C0F05D152EA03361CBF104683
:1003800019460AD181EA030101F0004141F0FE4122
:1003900041F470014FF0000070BD41F0FE4141F4A6
:1003A000780170BD81F0004102E000BF83F000439E
:1003B00030B54FEA41044FEA430594EA050F08BF00
:1003C00090EA020F1FBF54EA000C55EA020C7FEAC4
:1003D000645C7FEA655C00F0E2804FEA5454D4EB41
:1003E0005555B8BF6D420CDD2C4480EA020281EA0B
:1003F000030382EA000083EA010180EA020281EA43
:100400000303362D88BF30BD11F0004F4FEA013194
:100410004FF4801C4CEA113102D0404261EB4101A3
:1004200013F0004F4FEA03334CEA133302D0524229
:1004300063EB430394EA050F00F0A780A4F10104E5
:10044000D5F1200E0DDB02FA0EFC22FA05F280181F
:1004500041F1000103FA0EF2801843FA05F3594105
:100460000EE0A5F120050EF1200E012A03FA0EFC84
:1004700028BF4CF0020C43FA05F3C01851EBE371AE
:1004800001F0004507D54FF0000EDCF1000C7EEBCB
:1004900000006EEB0101B1F5801F1BD3B1F5001F09
:1004A0000CD349085FEA30004FEA3C0C04F1010428
:1004B0004FEA445212F5800F80F09A80BCF1004F51
:1004C00008BF5FEA500C50F1000041EB045141EAD3
:1004D000050130BD5FEA4C0C404141EB0101013C9C
:1004E00028BFB1F5801FE9D291F0000F04BF01468B
:1004F0000020B1FA81F308BF2033A3F10B03B3F15D
:1005000020020CDA0C3208DD02F1140CC2F10C02EC
:1005100001FA0CF021FA02F10CE002F11402D8BF4A
:10052000C2F1200C01FA02F120FA0CFCDCBF41EA16
:100530000C019040E41AA2BF01EB0451294330BDE5
:100540006FEA04041F3C1CDA0C340EDC04F11404C2
:10055000C4F1200220FA04F001FA02F340EA030099
:1005600021FA04F345EA030130BDC4F10C04C4F1DF
:10057000200220FA02F001FA04F340EA03002946BF
:1005800030BD21FA04F0294630BD94F0000F83F409
:10059000801306BF81F480110134013D4EE77FEAEC
:1005A000645C18BF7FEA655C29D094EA050F08BF38
:1005B00090EA020F05D054EA000C04BF1946104619
:1005C00030BD91EA030F1EBF0021002030BD5FEA5D
:1005D000545C05D14000494128BF41F0004130BD85
:1005E00014F580043CBF01F5801130BD01F00045D9
:1005F00045F0FE4141F470014FF0000030BD7FEA4C
:10060000645C1ABF194610467FEA655C1CBF0B4646
:10061000024650EA013406BF52EA033591EA030F5D
:1006200041F4002130BD00BF90F0000F04BF002155
:10063000704730B54FF4806404F132044FF0000588
:100640004FF0000150E700BF90F0000F04BF002101
:10065000704730B54FF4806404F1320410F0004567
:1006600048BF40424FF000013EE700BF42004FEA62
:10067000E2014FEA31014FEA02701FBF12F07F43DF
:1006800093F07F4F81F06051704732F07F4208BF96
:10069000704793F07F4F04BF41F40021704730B59D
:1006A0004FF4607401F0004521F000411CE700BFE9
:1006B00050EA010208BF704730B54FF000050AE06C
:1006C00050EA010208BF704730B511F0004502D56D
:1006D000404261EB41014FF4806404F132045FEA6F
:1006E000915C3FF4D8AE4FF003025FEADC0C18BF18
:1006F00003325FEADC0C18BF033202EBDC02C2F10A
:10070000200300FA03FC20FA02F001FA03FE40EA9B
:100710000E0021FA02F11444BDE600BF4FEA410287
:1007200012F5001215D211D56FF47873B3EB625243
:1007300012D94FEAC12343F0004343EA505311F06A
:10074000004F23FA02F018BF404270474FF00000FC
:10075000704750EA013005D111F0004008BF6FF03A
:10076000004070474FF00000704700BF00000000DD
:1007700080B586B000AF00F0FBFD00F0BDF800F0E2
:100780007FF900F0FFF800F02BF900F04BFA50A3CE
:10079000D3E90023C7E904230021002000F0AAFBCD
:1007A00001224D494D4800F03BFC1E21002000F085
:1007B000A1FB012248494A4800F032FC00F0F6FA59
:1007C0004FF47A7000F036FE0721002000F0B5F9F2
:1007D00040F6B83000F02EFE0721002000F0E3F9CB
:1007E00040F6B83000F026FE00F013FA00F03DFCB1
:1007F0000021002000F07EFB01223749394800F03B
:100800000FFCD7E90401FFF789FF0346FB60F86896
:10081000FFF71AFF02460B46D7E90401FFF7C6FDB2
:1008200002460B46104619464FF000022E4BFFF7CA
:100830008FFC02460B4610461946FFF76FFF034632
:10084000BB603B1D0A221946F86802F0E1FC3B46FA
:100850000A221946B86802F0DBFC1E21002000F0D5
:1008600049FB01221C49214800F0DAFB00F09EFA06
:100870001E21042000F03EFB3B1D012216491846B4
:1008800000F0CEFB1E21182000F034FB012212499B
:10089000174800F0C5FB1E21242000F02BFB3B462F
:1008A00001220D49184600F0BBFB1E213C2000F040
:1008B00021FB012208490F4800F0B2FB00F076FA54
:1008C0004FF4FA7000F0B6FD9BE700BFAFF3008075
:1008D0001F85EB51B89E44400000002008330008FB
:1008E0001033000818330008000059402433000872
:1008F000343300083833000880B590B000AF07F1FA
:10090000180328220021184602F0C6FC3B1D0022D5
:100910001A605A609A60DA601A610123BB614FF471
:100920008033FB6100233B620123BB6202237B63B4
:100930004FF48033BB634FF4E013FB6307F11803FC
:10094000184601F0E5FD0346002B01D000F0F0F859
:100950000F237B600223BB600023FB604FF48063A6
:100960003B6100237B613B1D0221184602F052F8D7
:100970000346002B01D000F0DBF800BF4037BD4636
:1009800080BD000080B500AF124B134A1A60114BB6
:10099000124A5A600F4B00229A600E4B0022DA6016
:1009A0000C4B4FF480421A610A4B00225A61094BEA
:1009B00000229A61074B0022DA61064B00221A627C
:1009C000044800F0DBFF0346002B01D000F0B0F834
:1009D00000BF80BD3000002000540040801A060097
:1009E00080B586B000AF07F1080300221A605A6094
:1009F0009A60DA603B4600221A605A601E4B1F4A1A
:100A00001A601D4B47225A601B4B00229A601A4BFA
:100A10004FF6FF72DA60184B00221A61164B002263
:100A20005A61154B00229A61134802F06DF9034692
:100A3000002B01D000F07CF84FF48053BB6007F12D
:100A4000080319460C4802F0AEF90346002B01D00A
:100A500000F06EF800233B6000237B603B461946A4
:100A6000054802F05FFB0346002B01D000F060F860
:100A700000BF1837BD4680BD84000020002C014017
:100A800080B588B000AF07F1100300221A605A60E9
:100A90009A60DA60244B9B69234A43F01003936108
:100AA000214B9B6903F01003FB60FB681E4B9B69A5
:100AB0001D4A43F0200393611B4B9B6903F0200305
:100AC000BB60BB68184B9B69174A43F004039361F2
:100AD000154B9B6903F004037B607B68124B9B6999
:100AE000114A43F0080393610F4B9B6903F008031D
:100AF0003B603B6800224FF400510C4800F026FF99
:100B00004FF400533B6101237B610023BB6102234F
:100B1000FB6107F110031946044800F093FD00BF84
:100B20002037BD4680BD00BF0010024000100140CC
:100B300080B400AF72B600BFFEE780B582B000AFF0
:100B400003460A46FB711346BB712622002178201A
:100B500000F00EFB00220021782000F009FBFB7959
:100B60001A460021782000F003FB002200217820A3
:100B700000F0FEFABB791A460021782000F0F8FA5E
:100B800000220021782000F0F3FAFF2200217820D3
:100B900000F0EEFA2F220021782000F0E9FA00BFE1
:100BA0000837BD4680BD80B582B000AF03460A4617
:100BB000FB711346BB7127220021782000F0D8FA80
:100BC00000220021782000F0D3FAFB791A46002198
:100BD000782000F0CDFA00220021782000F0C8FA39
:100BE000BB791A460021782000F0C2FA00220021C9
:100BF000782000F0BDFAFF220021782000F0B8FA3A
:100C00002F220021782000F0B3FA00BF0837BD463C
:100C100080BD80B500AF2E220021782000F0A8FA18
:100C200000BF80BD80B582B000AF00F027FA44F667
:100C30002063012278215B4801F0E2F80346002B93
:100C400001D00023A9E040F6C4137B6002E07B687A
:100C5000013B7B607B68002BF9D1AE22002178201C
:100C600000F086FA20220021782000F081FA10227C
:100C70000021782000F07CFAB0220021782000F0DA
:100C800077FAC8220021782000F072FA00220021B1
:100C9000782000F06DFA10220021782000F068FA28
:100CA00040220021782000F063FA81220021782080
:100CB00000F05EFAFF220021782000F059FAA1220C
:100CC0000021782000F054FAA6220021782000F0BC
:100CD0004FFAA8220021782000F04AFA3F22002192
:100CE000782000F045FAA4220021782000F040FA94
:100CF000D3220021782000F03BFA00220021782046
:100D000000F036FAD5220021782000F031FAF022E6
:100D10000021782000F02CFAD9220021782000F060
:100D200027FA22220021782000F022FADA2200217C
:100D3000782000F01DFA12220021782000F018FA25
:100D4000DB220021782000F013FA202200217820F5
:100D500000F00EFA8D220021782000F009FA14220A
:100D60000021782000F004FAAF220021782000F062
:100D7000FFF92E220021782000F0FAF9002000F07F
:100D800043F800F013F8084B00221A80064B0022AB
:100D90005A80054B01225A71012318460837BD4677
:100DA00080BD00BF30000020CC04002080B582B0A0
:100DB00000AF0023FB711DE0FB79503BDBB21A460C
:100DC0000021782000F0D4F900220021782000F0E2
:100DD000CFF910220021782000F0CAF9FB79DB015D
:100DE000084A1A4480234021782000F05BF9FB79FF
:100DF0000133FB71FB79072BDED900BF00BF083739
:100E0000BD4680BDCC00002080B582B000AF034657
:100E1000FB71FB79002B01D1002300E0FF234FF48D
:100E200080621946034802F037FA00BF0837BD4612
:100E300080BD00BFCC00002080B483B000AF03466B
:100E4000FB800B46BB801346FB70FB887F2B48D88A
:100E5000BB883F2B45D8254B1B79002B06D0FB7850
:100E6000002B0CBF01230023DBB2FB70FB78012BAE
:100E70001AD1FA88BB88DB0898B20346DB01134419
:100E80001B4AD35C5AB2BB8803F00703012101FA65
:100E900003F35BB2134359B2FA880346DB011344F0
:100EA000C9B2134AD1541DE0FA88BB88DB0898B256
:100EB0000346DB0113440E4AD35C5AB2BB8803F0ED
:100EC0000703012101FA03F35BB2DB435BB213407A
:100ED00059B2FA880346DB011344C9B2044AD1541B
:100EE00000E000BF0C37BD4680BC7047CC0400203A
:100EF000CC00002080B483B000AF03460A46FB80DC
:100F00001346BB80054AFB881380044ABB88538084
:100F100000BF0C37BD4680BC704700BFCC0400202A
:100F200080B586B000AF03463960FB711346BB71D4
:100F30003A4B1B881A463B681B7813447F2B07DC0F
:100F4000364B5B881A463B685B7813443F2B01DDC8
:100F500000235EE000237B614BE03B685A68FB792D
:100F6000203B3968497801FB03F319467B690B4440
:100F70005B0013441B88FB6000233B6130E0FA6890
:100F80003B6902FA03F303F40043002B10D0234B18
:100F90001A883B699BB2134498B2204B5A887B69EC
:100FA0009BB213449BB2BA791946FFF745FF14E090
:100FB0001A4B1A883B699BB2134498B2174B5A8854
:100FC0007B699BB2134499B2BB79002B0CBF012300
:100FD0000023DBB21A46FFF72FFF3B6901333B6169
:100FE0003B681B781A463B699342C8D37B6901333F
:100FF0007B613B685B781A467B699342ADD3074BB4
:101000001A883B681B789BB213449AB2034B1A8030
:10101000FB7918461837BD4680BD00BFCC040020C0
:1010200080B584B000AFF860B9601346FB7112E080
:10103000FB681B78FA79B9681846FFF771FF034619
:101040001A46FB681B789A4202D0FB681B7808E0BE
:10105000FB680133FB60FB681B78002BE8D1FB6861
:101060001B7818461037BD4680BD80B500AF002004
:10107000FFF7CAFEFFF79AFE00BF80BD80B483B0C1
:1010800000AF074B7B6002E07B68013B7B607B68C5
:10109000002BF9D100BF00BF0C37BD4680BC7047A4
:1010A00090D0030090B5C7B002AF0446084607F5DC
:1010B0008871A1F588710A60194607F58873A3F253
:1010C000091322461A7007F58873A3F58573024643
:1010D0001A7007F58873A3F586730A461A8007F518
:1010E0008873A3F5827307F58872A2F5857212786A
:1010F0001A70002387F80F3115E097F80F3107F5C4
:101100008872A2F5887212681A4497F80F31013379
:10111000117807F58872A2F58272D15497F80F31D1
:10112000013387F80F3197F80F319BB207F58872BA
:10113000A2F5867212889A42DFD807F58873A3F267
:1011400009131B7899B207F58873A3F586731B887A
:1011500001339BB207F10C020A200090034800F013
:1011600051FD00BF07F58A77BD4690BD30000020D5
:1011700080B586B002AF0346FB710B46BB711346C8
:101180007B71BB793B737B797B73FB7999B207F1F8
:101190000C020A2300930223034800F033FD00BF32
:1011A0001037BD4680BD00BF3000002080B485B040
:1011B00000AF154B9B69144A43F001039361124B36
:1011C0009B6903F00103BB60BB680F4BDB690E4AF0
:1011D00043F08053D3610C4BDB6903F080537B6099
:1011E0007B680A4B5B68FB60FB6823F0E063FB6095
:1011F000FB6843F00073FB60044AFB68536000BF68
:101200001437BD4680BC704700100240000001400A
:1012100080B588B000AF786007F1100300221A6033
:101220005A609A60DA607B681B68154A934223D142
:10123000144B9B69134A43F008039361114B9B695C
:1012400003F00803FB60FB68C0233B6112237B6152
:101250000323FB6107F1100319460B4800F0F2F974
:10126000084BDB69074A43F40013D361054BDB6984
:1012700003F40013BB60BB6800BF2037BD4680BDD0
:101280000054004000100240000C014080B485B0C2
:1012900000AF78607B681B68094A93420BD1094B09
:1012A0009B69084A43F400639361064B9B6903F40E
:1012B0000063FB60FB6800BF1437BD4680BC70470D
:1012C000002C01400010024080B400AFFEE780B463
:1012D00000AFFEE780B400AFFEE780B400AFFEE7EA
:1012E00080B400AFFEE780B400AF00BFBD4680BC55
:1012F000704780B400AF00BFBD4680BC704780B46B
:1013000000AF00BFBD4680BC704780B500AF00F0A5
:1013100075F800BF80BD80B400AF00BFBD4680BC83
:1013200070470000FFF7F7FF0B480C490C4A0023F9
:1013300002E0D458C4500433C4188C42F9D3094A8B
:10134000094C002301E013600432A242FBD301F0F8
:10135000ABFFFFF70DFA70470000002014000020DB
:10136000F440000814000020D8040020FEE700002C
:1013700080B500AF084B1B68074A43F010031360A9
:10138000032000F02BF90F2000F008F8FFF70EFF04
:101390000023184680BD00BF0020024080B582B007
:1013A00000AF7860124B1A68124B1B7819464FF445
:1013B0007A73B3FBF1F3B2FBF3F3184600F035F99F
:1013C0000346002B01D001230EE07B680F2B0AD8C7
:1013D000002279684FF0FF3000F00BF9064A7B6875
:1013E0001360002300E0012318460837BD4680BD86
:1013F00008000020100000200C00002080B400AF86
:10140000054B1B781A46054B1B681344034A1360AF
:1014100000BFBD4680BC704710000020D4040020EF
:1014200080B400AF024B1B681846BD4680BC7047B5
:10143000D404002080B584B000AF7860FFF7F0FFDF
:10144000B8607B68FB60FB68B3F1FF3F05D00A4BD7
:101450001B781A46FB681344FB6000BFFFF7E0FFF0
:101460000246BB68D31AFA689A42F7D800BF00BF99
:101470001037BD4680BD00BF1000002080B485B08D
:1014800000AF78607B6803F00703FB600C4BDB6800
:10149000BB60BA684FF6FF031340BB60FB681A02DB
:1014A000BB68134343F0BF6343F40033BB60044A9B
:1014B000BB68D36000BF1437BD4680BC704700BF17
:1014C00000ED00E080B400AF044BDB681B0A03F0C2
:1014D00007031846BD4680BC704700BF00ED00E022
:1014E00080B483B000AF03463960FB7197F90730D1
:1014F000002B0ADB3B68DAB20C4997F9073012017E
:10150000D2B20B4483F800230AE03B68DAB2084900
:10151000FB7903F00F03043B1201D2B20B441A769D
:1015200000BF0C37BD4680BC704700BF00E100E043
:1015300000ED00E080B489B000AFF860B9607A6077
:10154000FB6803F00703FB61FB69C3F10703042B8E
:1015500028BF0423BB61FB690433062B02D9FB6956
:10156000033B00E000237B614FF0FF32BB6902FACE
:1015700003F3DA43BB681A407B699A404FF0FF31AE
:101580007B6901FA03F3D9437B680B401343184688
:101590002437BD4680BC704780B582B000AF78600C
:1015A0007B68013BB3F1807F01D301230FE00A4A3E
:1015B0007B68013B53600F214FF0FF30FFF790FF36
:1015C000054B00229A60044B07221A60002318463C
:1015D0000837BD4680BD00BF10E000E080B582B096
:1015E00000AF78607868FFF749FF00BF0837BD4655
:1015F00080BD80B586B000AF0346B9607A60FB73EA
:1016000000237B61FFF75EFF78617A68B9687869CB
:10161000FFF790FF024697F90F3011461846FFF783
:101620005FFF00BF1837BD4680BD80B582B000AFF8
:1016300078607868FFF7B0FF034618460837BD4664
:1016400080BD000080B48BB000AF786039600023AB
:101650007B6200233B6269E101227B6A02FA03F3A9
:10166000FB613B681B68FA691340BB61BA69FB699F
:101670009A4240F058813B685B689A4A93425ED038
:10168000984A934275D8984A934258D0964A9342C2
:101690006FD8964A934252D0944A934269D8944A5A
:1016A00093424CD0924A934263D8924A934246D096
:1016B000904A93425DD8122B2AD8122B59D801A2F6
:1016C00052F823F03F170008191700082B170008DD
:1016D0006D170008731700087317000873170008C8
:1016E00073170008731700087317000873170008B2
:1016F00073170008731700087317000873170008A2
:101700007317000873170008211700083517000821
:10171000794A934213D02CE03B68DB683B6229E0B6
:101720003B68DB6804333B6224E03B68DB680833DA
:101730003B621FE03B68DB680C333B621AE03B68AE
:101740009B68002B02D104233B6213E03B689B683B
:10175000012B05D108233B627B68FA691A6109E015
:1017600008233B627B68FA695A6103E000233B620D
:1017700000E000BFBB69FF2B01D87B6801E07B68FC
:1017800004337B61BB69FF2B02D87B6A9B0002E0BC
:101790007B6A083B9B003B617B691A680F213B69B0
:1017A00001FA03F3DB431A40396A3B6901FA03F398
:1017B0001A437B691A603B685B6803F08053002B17
:1017C00000F0B1804D4B9B694C4A43F0010393619B
:1017D0004A4B9B6903F00103BB60BB68484A7B6AC4
:1017E0009B08023352F82330FB607B6A03F003034B
:1017F0009B000F2202FA03F3DB43FA681340FB60FD
:101800007B68404A934213D07B683F4A93420DD095
:101810007B683E4A934207D07B683D4A934201D1A0
:10182000032306E0042304E0022302E0012300E096
:1018300000237A6A02F0030292009340FA6813438D
:10184000FB602F497B6A9B080233FA6841F823202A
:101850003B685B6803F48013002B06D02D4B9A681D
:101860002C49BB6913438B6006E02A4B9A68BB691D
:10187000DB43284913408B603B685B6803F400132B
:10188000002B06D0234BDA682249BB691343CB6097
:1018900006E0204BDA68BB69DB431E491340CB608E
:1018A0003B685B6803F40033002B06D0194B5A6881
:1018B0001849BB6913434B6006E0164B5A68BB6975
:1018C000DB43144913404B603B685B6803F480338F
:1018D000002B21D00F4B1A680E49BB6913430B60D4
:1018E00021E000BF00003210000031100000221083
:1018F0000000211000001210000011100010024022
:101900000000014000080140000C014000100140AF
:1019100000140140000401400B4B1A68BB69DB4313
:10192000094913400B607B6A01337B623B681A688C
:101930007B6A22FA03F3002B7FF48EAE00BF00BF58
:101940002C37BD4680BC70470004014080B483B092
:1019500000AF78600B467B8013467B707B78002B52
:1019600003D07A887B681A6103E07B881A047B685D
:101970001A6100BF0C37BD4680BC704780B584B08B
:1019800000AF78607B68002B01D101232BE17B68DD
:1019900093F83D30DBB2002B06D17B68002283F840
:1019A0003C207868FFF734FC7B68242283F83D20D4
:1019B0007B681B681A687B681B6822F001021A604A
:1019C0007B681B681A687B681B6842F400421A60D7
:1019D0007B681B681A687B681B6822F400421A60E7
:1019E00001F060F9F8607B685B68814A934207D830
:1019F000FB68804A934294BF01230023DBB206E0D8
:101A0000FB687D4A934294BF01230023DBB2002B85
:101A100001D00123E7E0FB68784AA2FB03239B0C7B
:101A2000BB607B681B685B6823F03F017B681B68B9
:101A3000BA680A435A607B681B681B6A23F03F013F
:101A40007B685B686A4A934202D8BB68013309E04D
:101A5000BB684FF4967202FB03F3694AA2FB0323AF
:101A60009B0901337A6812680B4313627B681B6819
:101A7000DB6923F44F4222F0FF027B685B685C491C
:101A80008B4219D8FB68591E7B685B685B00B1FB11
:101A9000F3F3591C40F6FC730B40002B0AD0FB6893
:101AA000591E7B685B685B00B1FBF3F30133C3F342
:101AB0000B0351E004234FE07B689B68002B11D19E
:101AC000FB68581E7B6859680B465B000B44B0FBF3
:101AD000F3F30133C3F30B03002B0CBF01230023EB
:101AE000DBB212E0FB68581E7B6859680B469B000E
:101AF0000B4499000B44B0FBF3F30133C3F30B0326
:101B0000002B0CBF01230023DBB2002B01D00123EB
:101B100022E07B689B68002B0ED1FB68581E7B6817
:101B200059680B465B000B44B0FBF3F30133C3F37E
:101B30000B0343F400430FE0FB68581E7B685968B1
:101B40000B469B000B4499000B44B0FBF3F30133AD
:101B5000C3F30B0343F44043796809681343CB6133
:101B60007B681B681B6823F0C0017B68DA697B68AF
:101B70001B6A1A437B681B680A431A607B681B68F0
:101B80009B6823F4034323F0FF037A6811697A68A2
:101B9000D26811437A6812680B4393607B681B68B4
:101BA000DB6823F0FF017B685A697B689B691A43F5
:101BB0007B681B680A43DA607B681B681A687B686D
:101BC0001B6842F001021A607B6800221A647B687D
:101BD000202283F83D207B6800221A637B68002264
:101BE00083F83E20002318461037BD4680BD00BF55
:101BF000A08601007F841E00FF083D0083DE1B439A
:101C0000D34D621080B588B002AFF8607A601A4692
:101C10000B467B8113463B81FFF702FC7861FB6832
:101C200093F83D30DBB2202B40F0E0807B690093DD
:101C3000192301227049F86800F092FA0346002B3C
:101C400001D00223D3E0FB6893F83C30012B01D193
:101C50000223CCE0FB68012283F83C20FB681B6870
:101C60001B6803F00103012B07D0FB681B681A688F
:101C7000FB681B6842F001021A60FB681B681A6867
:101C8000FB681B6822F400621A60FB68212283F85B
:101C90003D20FB68102283F83E20FB6800221A6476
:101CA000FB687A685A62FB683A895A85FB685B8DE3
:101CB0009AB2FB681A85FB68504ADA6279897B69B7
:101CC0003A6AF86800F0CAF90346002B01D00123F4
:101CD0008DE000233B61FB681B685B693B61FB682F
:101CE0001B689B693B613B6966E07A69396AF86801
:101CF00000F050FB0346002B0DD0FB681B6C042B3F
:101D000007D1FB681B681A68FB681B6842F4007205
:101D10001A6001236BE0FB685B6A1A78FB681B683A
:101D20001A61FB685B6A5A1CFB685A62FB685B8D30
:101D30009BB2013B9AB2FB685A85FB681B8D013B45
:101D40009AB2FB681A85FB681B685B6903F00403A1
:101D5000042B1BD1FB681B8D002B17D0FB685B6A23
:101D60001A78FB681B681A61FB685B6A5A1CFB687F
:101D70005A62FB685B8D9BB2013B9AB2FB685A8545
:101D8000FB681B8D013B9AB2FB681A857A69396A38
:101D9000F86800F047FB0346002B0DD0FB681B6C76
:101DA000042B07D1FB681B681A68FB681B6842F4A8
:101DB00000721A6001231AE0FB681B8D002B94D17E
:101DC000FB681B681A68FB681B6842F400721A60A3
:101DD000FB68202283F83D20FB68002283F83E2028
:101DE000FB68002283F83C20002300E00223184611
:101DF0001837BD4680BD00BF020010000000FFFF85
:101E000080B58AB002AFF8607A603B600B467B8198
:101E1000FFF706FBF8610023BB61FB6893F83D30D8
:101E2000DBB2202B40F01181FB69009319230122C2
:101E30008849F86800F094F90346002B01D002238A
:101E400004E1FB6893F83C30012B01D10223FDE053
:101E5000FB68012283F83C20FB681B681B6803F0C9
:101E60000103012B07D0FB681B681A68FB681B681D
:101E700042F001021A60FB681B681A68FB681B6865
:101E800022F400621A60FB68242283F83D20FB687C
:101E900000221A64FB68704ADA62FB681B681A68E1
:101EA000FB681B6842F480721A60FB6900933B6810
:101EB00000224FF00111F86800F052F90346002BA0
:101EC0000DD0FB681B681B6803F48073B3F5807F3B
:101ED00003D1FB684FF400721A640323B6E07B89D8
:101EE000DBB21A46FB681B6802F0FE021A61FFF7BC
:101EF00097FAF861FB681B685B6903F00203022B29
:101F00000CBF01230023DBB2FB75FB681B685B6918
:101F100003F48063B3F5806F0CBF01230023DBB2B1
:101F2000BB7525E0FFF77CFA0246FB69D31A3A68D5
:101F30009A4202D33B68002B03D1FB68A02283F8AE
:101F40003D20FB681B685B6903F00203022B0CBF9A
:101F500001230023DBB2FB75FB681B685B6903F49C
:101F60008063B3F5806F0CBF01230023DBB2BB7528
:101F7000FB6893F83D30DBB2A02B05D0FB7D002B36
:101F800002D1BB7D002BCDD0FB68202283F83D2001
:101F9000FB681B685B6903F00203022B29D1FB6815
:101FA0001B681A68FB681B6842F400721A60002301
:101FB0003B61FB681B685B693B61FB681B689B6955
:101FC0003B613B69FB690093192301222149F868B1
:101FD00000F0C6F80346002B01D0012336E0FB6871
:101FE000202283F83D20FB68002283F83C20002358
:101FF0002CE0FB681B681A68FB681B6842F40072DF
:102000001A60FB681B686FF480625A61FB69009379
:10201000192301220F49F86800F0A2F80346002BAB
:1020200001D0012312E0BB690133BB61BA697B684F
:102030009A42FFF432AFFB68202283F83D20FB6810
:10204000002283F83C20012300E0022318462037B9
:10205000BD4680BD020010000000FFFF80B588B0C3
:1020600002AFF8607A603B600B467B81FB68DB6AFD
:102070007B617B69082B06D07B69012B03D07B69D0
:1020800013F5803F08D1FB681B681A68FB681B6862
:1020900042F480721A600BE0FB681B6B122B07D1B5
:1020A000FB681B681A68FB681B6842F480721A6040
:1020B0003B6800937B6800224FF00111F86800F044
:1020C0004FF80346002B0DD0FB681B681B6803F418
:1020D0008073B3F5807F03D1FB684FF400721A64FC
:1020E000032335E0FB681B69B3F5804F08D17B897A
:1020F000DBB21A46FB681B6802F0FE021A611BE0A5
:102100007B89DB11DBB203F00603DBB263F00F0364
:10211000DAB2FB681B681A613B687A680E49F86896
:1021200000F098F80346002B01D0012310E07B89D2
:10213000DAB2FB681B681A613B687A680749F8687D
:1021400000F088F80346002B01D0012300E00023B3
:1021500018461837BD4680BD080001000200010086
:1021600080B584B000AFF860B9603B601346FB7186
:1021700048E03B68B3F1FF3F44D0FFF751F9024616
:10218000BB69D31A3A689A4202D33B68002B39D113
:10219000BB681B0CDBB2012B0DD1FB681B685B69B4
:1021A000DA43BB6813409BB2002B0CBF0123002312
:1021B000DBB21A460CE0FB681B689B69DA43BB681C
:1021C00013409BB2002B0CBF01230023DBB21A4645
:1021D000FB799A4216D1FB6800221A63FB68202221
:1021E00083F83D20FB68002283F83E20FB681B6CCF
:1021F00043F02002FB681A64FB68002283F83C204D
:10220000012323E0BB681B0CDBB2012B0DD1FB6863
:102210001B685B69DA43BB6813409BB2002B0CBFA1
:1022200001230023DBB21A460CE0FB681B689B69A4
:10223000DA43BB6813409BB2002B0CBF0123002381
:10224000DBB21A46FB799A4293D000231846103726
:10225000BD4680BD80B584B000AFF860B9607A60DB
:102260003B6071E0FB681B685B6903F48063B3F556
:10227000806F23D1FB681B681A68FB681B6842F4F7
:1022800000721A60FB681B686FF480625A61FB6819
:1022900000221A63FB68202283F83D20FB6800229D
:1022A00083F83E20FB681B6C43F00402FB681A6451
:1022B000FB68002283F83C20012367E07B68B3F1D0
:1022C000FF3F41D0FFF7ACF802463B68D31A7A686B
:1022D0009A4202D37B68002B36D1BB681B0CDBB261
:1022E000012B0CD1FB681B685B69DA43BB681340A8
:1022F0009BB2002B14BF01230023DBB20BE0FB6871
:102300001B689B69DA43BB6813409BB2002B14BF68
:1023100001230023DBB2002B16D0FB6800221A63D6
:10232000FB68202283F83D20FB68002283F83E20D2
:10233000FB681B6C43F02002FB681A64FB680022F8
:1023400083F83C20012321E0BB681B0CDBB2012B8E
:102350000CD1FB681B685B69DA43BB6813409BB216
:10236000002B14BF01230023DBB20BE0FB681B68CA
:102370009B69DA43BB6813409BB2002B14BF012357
:102380000023DBB2002B7FF46DAF0023184610371B
:10239000BD4680BD80B584B000AFF860B9607A609A
:1023A00034E0F86800F086F80346002B01D00123E2
:1023B00034E0BB68B3F1FF3F28D0FFF731F80246A5
:1023C0007B68D31ABA689A4202D3BB68002B1DD12E
:1023D000FB681B685B6903F08003802B16D0FB68E9
:1023E00000221A63FB68202283F83D20FB6800224C
:1023F00083F83E20FB681B6C43F02002FB681A64E4
:10240000FB68002283F83C20012307E0FB681B687F
:102410005B6903F08003802BC3D10023184610377B
:10242000BD4680BD80B584B000AFF860B9607A6009
:1024300034E0F86800F03EF80346002B01D0012399
:1024400034E0BB68B3F1FF3F28D0FEF7E9FF024656
:102450007B68D31ABA689A4202D3BB68002B1DD19D
:10246000FB681B685B6903F00403042B16D0FB6850
:1024700000221A63FB68202283F83D20FB680022BB
:1024800083F83E20FB681B6C43F02002FB681A6453
:10249000FB68002283F83C20012307E0FB681B68EF
:1024A0005B6903F00403042BC3D1002318461037E3
:1024B000BD4680BD80B483B000AF78607B681B6888
:1024C0005B6903F48063B3F5806F1BD17B681B6885
:1024D0006FF480625A617B6800221A637B68202255
:1024E00083F83D207B68002283F83E207B681B6CCC
:1024F00043F004027B681A647B68002283F83C2066
:10250000012300E0002318460C37BD4680BC70470D
:1025100080B586B000AF78607B68002B01D10123C5
:1025200072E27B681B6803F00103002B00F08780D8
:10253000924B5B6803F00C03042B0CD08F4B5B6851
:1025400003F00C03082B12D18C4B5B6803F480332F
:10255000B3F5803F0BD1894B1B6803F40033002B8C
:102560006CD07B685B68002B68D101234CE27B68F0
:102570005B68B3F5803F06D1804B1B687F4A43F40C
:10258000803313602EE07B685B68002B0CD17B4BA3
:102590001B687A4A23F480331360784B1B68774AB0
:1025A00023F4802313601DE07B685B68B3F5A02FE4
:1025B0000CD1724B1B68714A43F4802313606F4B3C
:1025C0001B686E4A43F4803313600BE06B4B1B684F
:1025D0006A4A23F480331360684B1B68674A23F40C
:1025E000802313607B685B68002B13D0FEF718FF15
:1025F000386108E0FEF714FF02463B69D31A642BEA
:1026000001D9032300E25D4B1B6803F40033002B68
:10261000F0D014E0FEF704FF386108E0FEF700FF99
:1026200002463B69D31A642B01D90323ECE1534BD7
:102630001B6803F40033002BF0D100E000BF7B687F
:102640001B6803F00203002B63D04C4B5B6803F064
:102650000C03002B0BD0494B5B6803F00C03082BD9
:102660001CD1464B5B6803F48033002B16D1434BDF
:102670001B6803F00203002B05D07B681B69012B4C
:1026800001D00123C0E13D4B1B6823F0F8027B68B9
:102690005B69DB00394913430B603AE07B681B69D7
:1026A000002B20D0364B01221A60FEF7B9FE3861AC
:1026B00008E0FEF7B5FE02463B69D31A022B01D9AA
:1026C0000323A1E12D4B1B6803F00203002BF0D084
:1026D0002A4B1B6823F0F8027B685B69DB00274903
:1026E00013430B6015E0264B00221A60FEF798FE9C
:1026F000386108E0FEF794FE02463B69D31A022BCC
:1027000001D9032380E11D4B1B6803F00203002B5A
:10271000F0D17B681B6803F00803002B3AD07B687C
:102720009B69002B19D0174B01221A60FEF778FE27
:10273000386108E0FEF774FE02463B69D31A022BAB
:1027400001D9032360E10D4B5B6A03F00203002B08
:10275000F0D0012000F0BAFA1CE00A4B00221A6007
:10276000FEF75EFE38610FE0FEF75AFE02463B6957
:10277000D31A022B08D9032346E100BF0010024000
:102780000000424280044242924B5B6A03F0020323
:10279000002BE9D17B681B6803F00403002B00F0D9
:1027A000A6800023FB758B4BDB6903F08053002B65
:1027B0000DD1884BDB69874A43F08053D361854B49
:1027C000DB6903F08053BB60BB680123FB75824B60
:1027D0001B6803F48073002B18D17F4B1B687E4A63
:1027E00043F480731360FEF71BFE386108E0FEF7C8
:1027F00017FE02463B69D31A642B01D9032303E178
:10280000754B1B6803F48073002BF0D07B68DB688A
:10281000012B06D16F4B1B6A6E4A43F00103136212
:102820002DE07B68DB68002B0CD16A4B1B6A694A80
:1028300023F001031362674B1B6A664A23F004030B
:1028400013621CE07B68DB68052B0CD1614B1B6AB3
:10285000604A43F0040313625E4B1B6A5D4A43F017
:10286000010313620BE05B4B1B6A5A4A23F001031E
:102870001362584B1B6A574A23F0040313627B68A8
:10288000DB68002B15D0FEF7CBFD38610AE0FEF7C0
:10289000C7FD02463B69D31A41F28832934201D9FF
:1028A0000323B1E04B4B1B6A03F00203002BEED075
:1028B00014E0FEF7B5FD38610AE0FEF7B1FD02460F
:1028C0003B69D31A41F28832934201D903239BE03A
:1028D000404B1B6A03F00203002BEED1FB7D012B62
:1028E00005D13C4BDB693B4A23F08053D3617B68C5
:1028F000DB69002B00F08780364B5B6803F00C032C
:10290000082B61D07B68DB69022B46D1334B002258
:102910001A60FEF785FD386108E0FEF781FD02468A
:102920003B69D31A022B01D903236DE0294B1B68A5
:1029300003F00073002BF0D17B681B6AB3F5803F76
:1029400008D1244B5B6823F400327B689B682149E3
:1029500013434B601F4B5B6823F474127B68196A46
:102960007B685B6A0B431B4913434B601B4B012283
:102970001A60FEF755FD386108E0FEF751FD02468A
:102980003B69D31A022B01D903233DE0114B1B688D
:1029900003F00073002BF0D035E0104B00221A60DA
:1029A000FEF73EFD386108E0FEF73AFD02463B695E
:1029B000D31A022B01D9032326E0064B1B6803F030
:1029C0000073002BF0D11EE07B68DB69012B07D17F
:1029D000012319E0001002400070004060004242F4
:1029E0000B4B5B68FB60FB6803F480327B681B6AFF
:1029F0009A4206D1FB6803F470127B685B6A9A42C4
:102A000001D0012300E0002318461837BD4680BDE1
:102A10000010024080B584B000AF786039607B68F8
:102A2000002B01D10123D0E06A4B1B6803F00703A0
:102A30003A689A4210D9674B1B6823F00702654930
:102A40003B6813430B60634B1B6803F007033A6852
:102A50009A4201D00123B8E07B681B6803F00203AF
:102A6000002B20D07B681B6803F00403002B05D0EB
:102A7000594B5B68584A43F4E06353607B681B68BA
:102A800003F00803002B05D0534B5B68524A43F414
:102A900060535360504B5B6823F0F0027B689B6887
:102AA0004D4913434B607B681B6803F00103002B07
:102AB00040D07B685B68012B07D1474B1B6803F450
:102AC0000033002B15D101237FE07B685B68022B6C
:102AD00007D1414B1B6803F00073002B09D1012380
:102AE00073E03D4B1B6803F00203002B01D101236F
:102AF0006BE0394B5B6823F003027B685B68364907
:102B000013434B60FEF78CFCF8600AE0FEF788FC8C
:102B10000246FB68D31A41F28832934201D903235B
:102B200053E02D4B5B6803F00C027B685B689B00F5
:102B30009A42EBD1274B1B6803F007033A689A428D
:102B400010D2244B1B6823F0070222493B68134331
:102B50000B60204B1B6803F007033A689A4201D0D0
:102B6000012332E07B681B6803F00403002B08D0CC
:102B7000194B5B6823F4E0627B68DB6816491343FA
:102B80004B607B681B6803F00803002B09D0124BD5
:102B90005B6823F460527B681B69DB000E491343BA
:102BA0004B6000F021F802460B4B5B681B0903F0F9
:102BB0000F030A49CB5C22FA03F3094A1360094B5D
:102BC0001B681846FEF7EAFB002318461037BD467F
:102BD00080BD00BF00200240001002409C40000861
:102BE000080000200C00002080B487B000AF002354
:102BF000FB600023BB6000237B6100237B6000231C
:102C00003B611E4B5B68FB60FB6803F00C03042B0D
:102C100002D0082B03D027E0194B3B6127E0FB686B
:102C20009B0C03F00F03174AD35C7B60FB6803F433
:102C30008033002B10D0114B5B685B0C03F0010359
:102C4000114AD35CBB607B680D4A03FB02F2BB6890
:102C5000B2FBF3F37B6104E07B680C4A02FB03F3F5
:102C60007B617B693B6102E0054B3B6100BF3B69D7
:102C700018461C37BD4680BC704700BF001002409C
:102C800000127A00B4400008C440000800093D006A
:102C900080B400AF024B1B681846BD4680BC70472D
:102CA0000800002080B500AFFFF7F2FF0246054B99
:102CB0005B681B0A03F007030349CB5C22FA03F3AA
:102CC000184680BD00100240AC40000880B485B0BA
:102CD00000AF78600A4B1B680A4AA2FB03235B0A19
:102CE0007A6802FB03F3FB6000BFFB685A1EFA60C0
:102CF000002BF9D100BF00BF1437BD4680BC704720
:102D000008000020D34D621080B582B000AF78601B
:102D10007B68002B01D1012341E07B6893F83D30B3
:102D2000DBB2002B06D17B68002283F83C20786858
:102D3000FEF7ACFA7B68022283F83D207B681A68B4
:102D40007B6804331946104600F0F4F87B680122D2
:102D500083F846207B68012283F83E207B680122AD
:102D600083F83F207B68012283F840207B680122A2
:102D700083F841207B68012283F842207B6801228E
:102D800083F843207B68012283F844207B6801227A
:102D900083F845207B68012283F83D2000231846F4
:102DA0000837BD4680BD80B584B000AF786039601B
:102DB0000023FB737B6893F83C30012B01D1022385
:102DC000B4E07B68012283F83C207B68022283F810
:102DD0003D207B681B689B68BB60BB6823F0770362
:102DE000BB60BB6823F47F43BB607B681B68BA6829
:102DF0009A603B681B68B3F5005F3ED0B3F5005F97
:102E000000F28780B3F5805F00F08680B3F5805FC5
:102E10007FD8702B1AD0702B7BD8602B50D0602BB2
:102E200077D8502B3CD0502B73D8402B58D0402B08
:102E30006FD8302B64D0302B6BD8202B60D0202B58
:102E400067D8002B5CD0102B5AD062E07B681868E2
:102E50003B6899683B685A683B68DB6800F043F957
:102E60007B681B689B68BB60BB6843F07703BB60F3
:102E70007B681B68BA689A604FE07B6818683B689B
:102E800099683B685A683B68DB6800F02CF97B68FE
:102E90001B689A687B681B6842F480429A603CE039
:102EA0007B6818683B6859683B68DB681A4600F025
:102EB000A3F87B681B685021184600F0FAF82CE054
:102EC0007B6818683B6859683B68DB681A4600F005
:102ED000C1F87B681B686021184600F0EAF81CE026
:102EE0007B6818683B6859683B68DB681A4600F0E5
:102EF00083F87B681B684021184600F0DAF80CE084
:102F00007B681A683B681B681946104600F0D1F8C8
:102F100003E00123FB7300E000BF7B68012283F81C
:102F20003D207B68002283F83C20FB7B184610374D
:102F3000BD4680BD80B485B000AF786039607B68E5
:102F40001B68FB607B68294A93420BD07B68B3F116
:102F5000804F07D07B68264A934203D07B68254A7E
:102F6000934208D1FB6823F07003FB603B685B6809
:102F7000FA681343FB607B681C4A93420BD07B6862
:102F8000B3F1804F07D07B68194A934203D07B6826
:102F9000184A934208D1FB6823F44073FB603B68F6
:102FA000DB68FA681343FB60FB6823F080023B6830
:102FB0005B691343FB607B68FA681A603B689A6838
:102FC0007B68DA623B681A687B689A627B68074AAA
:102FD000934203D13B681A697B681A637B680122BC
:102FE0005A6100BF1437BD4680BC7047002C0140B9
:102FF000000400400008004080B487B000AFF860D3
:10300000B9607A60FB681B6A7B61FB681B6A23F00E
:103010000102FB681A62FB689B693B613B6923F014
:10302000F0033B617B681B013A6913433B617B6999
:1030300023F00A037B617A69BB6813437B61FB68F9
:103040003A699A61FB687A691A6200BF1C37BD460B
:1030500080BC704780B487B000AFF860B9607A6018
:10306000FB681B6A7B61FB681B6A23F01002FB682C
:103070001A62FB689B693B613B6923F470433B61C7
:103080007B681B033A6913433B617B6923F0A00310
:103090007B61BB681B017A6913437B61FB683A69FA
:1030A0009A61FB687A691A6200BF1C37BD4680BC12
:1030B000704780B485B000AF786039607B689B68EA
:1030C000FB60FB6823F07003FB603A68FB68134306
:1030D00043F00703FB607B68FA689A6000BF14370F
:1030E000BD4680BC704780B487B000AFF860B9605F
:1030F0007A603B60FB689B687B617B6923F47F435C
:103100007B613B681A027B681A43BB6813437A6988
:1031100013437B61FB687A699A6000BF1C37BD4628
:1031200080BC704780B485B000AF786039607B6840
:1031300093F83C30012B01D1022346E07B68012249
:1031400083F83C207B68022283F83D207B681B6863
:103150005B68FB607B681B689B68BB60FB6823F057
:103160007003FB603B681B68FA681343FB607B6875
:103170001B68FA685A607B681B68164A93420ED037
:103180007B681B68B3F1804F09D07B681B68124ACB
:10319000934204D07B681B68104A93420CD1BB68F1
:1031A00023F08003BB603B685B68BA681343BB6075
:1031B0007B681B68BA689A607B68012283F83D20AF
:1031C0007B68002283F83C20002318461437BD4654
:1031D00080BC7047002C0140000400400008004003
:1031E000931E222B10B50C4604D900231C460B70ED
:1031F000204610BD0A2A09D1002807DA2D230B70BA
:1032000001214042214400F005F8F1E70021F9E7EF
:10321000FFF7E6BFF0B58BB005460B466E461D4C7A
:1032200004F1200C374620686168083403C7644500
:103230003E46F7D1217920683971911E22293860E4
:103240004FF0000104D919700B4618460BB0F0BDC1
:10325000581E8446B5FBF2F702FB175628366E441B
:1032600016F8286C0C460CF8016F2E46B2423D460B
:1032700001F10101EED900225A541919A51AAA42E6
:10328000E3DA10F8015F0E780132067001F8015997
:10329000F4E700BFC640000803460244934200D151
:1032A000704703F8011BF9E770B500260C4D0D4C73
:1032B000641BA410A64209D100F01AF800260A4D9A
:1032C0000A4C641BA410A64205D170BD55F8043BFE
:1032D00098470136EEE755F8043B98470136F2E788
:1032E000EC400008EC400008EC400008F04000080A
:1032F000F8B500BFF8BC08BC9E467047F8B500BFE3
:08330000F8BC08BC9E467047B2
:103308004B6576696E00000054686F6E79000000A6
:1033180054656D7065726174757265002020202097
:103328002020202020202020200000002C00000049
:10333800646567726573000000000000000000000B
:103348000000000000000000000000000000000075
:103358000000000000000000000000000000000C59
:10336800000C000C000C000C000C000C000C000CF5
:10337800000C000C0000000C000C00000000000015
:103388000000001B001B001B001B001B00000000AE
:103398000000000000000000000000000000000025
:1033A8000000000000008019801980198019C07F72
:1033B800C07F80190033C07FC07F003300330033E3
:1033C80000330000000000000000001E003F807570
:1033D80080650074003C001E0007800580658065DC
:1033E8008075003F001E000400040000000000700B
:1033F80000D840D8C0D880D900730006000C801BC4
:10340800C036C066C046C006800300000000000049
:103418000000001E003F003300330033001E000C84
:10342800C03CC066806380618063C03E801C000031
:10343800000000000000000C000C000C000C000C48
:103448000000000000000000000000000000000074
:1034580000000000000000008000000100030006DA
:1034680000060004000C000C000C000C000C000C02
:103478000004000600060003000180000020001080
:103488000018000C000C00040006000600060006E8
:10349800000600060004000C000C001800100020B4
:1034A8000000000C002D003F001E0033000000004B
:1034B8000000000000000000000000000000000004
:1034C80000000000000000000000000C000C000CD0
:1034D800000CC0FFC0FF000C000C000C000C00002A
:1034E80000000000000000000000000000000000D4
:1034F80000000000000000000000000000000000C4
:103508000000000C000C000400040008000000008B
:103518000000000000000000000000000000001E85
:10352800001E000000000000000000000000000075
:103538000000000000000000000000000000000083
:1035480000000000000000000000000C000C00005B
:10355800000000000000000300030003000600064E
:1035680000060006000C000C000C000C00180018E7
:1035780000180000000000000000001E003F00339B
:10358800806180618061806D806D80618061806113
:103598000033003F001E000000000000000000068D
:1035A800000E001E00360026000600060006000673
:1035B80000060006000600060006000000000000E5
:1035C8000000001E003F807380618061800100035D
:1035D8000006000C001800300060807F807F00002B
:1035E800000000000000001C003E006300630003B0
:1035F800000E000E00038001800180618073003F8F
:10360800001E00000000000000000006000E000E72
:10361800001E001E0016003600360066807F807F80
:103628000006000600060000000000000000007F01
:10363800007F006000600060006E007F8063800192
:10364800800180618073003F001E000000000000C0
:103658000000001E003F803380610060006E007F24
:1036680080738061806180618033003F001E0000AC
:10367800000000000000807F807F800100030003BD
:1036880000060006000C000C000C000800180018CA
:1036980000180000000000000000001E003F8063CA
:1036A800806180610021001E003F8061806180612F
:1036B8008061003F001E0000000000000000001EA6
:1036C800003F00738061806180618073803F801D4E
:1036D800800180610073003F001E000000000000B0
:1036E80000000000000000000000000C000C0000BA
:1036F80000000000000000000000000C000C0000AA
:1037080000000000000000000000000000000000B1
:10371800000C000C00000000000000000000000C7D
:10372800000C000400040008000000000000000075
:1037380080008003000E003800600038000E80030F
:1037480080000000000000000000000000000000F1
:10375800000000000000807F807F00000000807F64
:10376800807F000000000000000000000000000052
:10377800000000000000000000400070001C00076E
:1037880080010007001C00700040000000000000DD
:10379800000000000000001F803FC071C060C00032
:1037A800C00180030007000E000C000C0000000C94
:1037B800000C0000000000000000001E003F8031E7
:1037C80080718063806F806D806D806F806700601E
:1037D8000032003E001C0000000000000000000E47
:1037E800000E001B001B001B001B80318031803F36
:1037F800803F8031C060C060C060000000000000F1
:103808000000007C007E0063006300630063007EAC
:10381800007E0063806180618063007F007E00001D
:10382800000000000000001E003F80318061006041
:103838000060006000600060006080618031003FCF
:10384800001E0000000000000000007C007F0063F4
:1038580080638061806180618061806180610063D4
:103868000063007E007C0000000000000000807FF4
:10387800807F0060006000600060007F007F006063
:10388800006000600060807F807F00000000000012
:103898000000807F807F0060006000600060007F23
:1038A800007F006000600060006000600060000051
:1038B800000000000000001E003F803180610060B1
:1038C8000060006080638063806180618031803F38
:1038D800001E00000000000000008061806180611F
:1038E800806180618061807F807F8061806180618C
:1038F8008061806180610000000000000000003FDE
:10390800003F000C000C000C000C000C000C000C1C
:10391800000C000C000C003F003F000000000000FD
:103928000000800180018001800180018001800108
:1039380080018001806180618073003F001E00006B
:10394800000000000000C06080610063006600663F
:10395800006C0078007C006600660063806180610E
:10396800C06000000000000000000060006000600F
:10397800006000600060006000600060006000603F
:103988000060807F807F0000000000000000C071A0
:10399800C071C07BC07AC06AC06AC06EC064C060B3
:1039A800C060C060C060C060C0600000000000006F
:1039B800000080718071807980798079806D806D58
:1039C800806D8065806780678067806380630000A2
:1039D800000000000000001E003F0033806180618D
:1039E8008061806180618061806180610033003F17
:1039F800001E0000000000000000007E007F8063C1
:103A08008061806180618063007F007E006000606B
:103A18000060006000600000000000000000001E60
:103A2800003F0033806180618061806180618061D6
:103A3800806580670033803F401E00000000000062
:103A48000000007E007F8063806180618063007F6A
:103A5800007E00660063006380618061C0600000D2
:103A6800000000000000000E001F8031803100308F
:103A78000038001E00078003806180618031003FAC
:103A8800001E0000000000000000C0FFC0FF000C86
:103A9800000C000C000C000C000C000C000C000CBE
:103AA800000C000C000C0000000000000000806109
:103AB80080618061806180618061806180618061F6
:103AC800806180618073003F001E000000000000DC
:103AD8000000C060C060C060803180318031001B50
:103AE800001B001B001B000E000E000E000400004F
:103AF800000000000000C0C0C0C0C0C0C0C0C0C03E
:103B0800C0CC804C804C805E805280528073806133
:103B180080610000000000000000C0C0806080617B
:103B28000033003B001E000C000C001E001F003B71
:103B380080718061C0C00000000000000000C0C0AB
:103B48008061806100330033001E001E000C000CF1
:103B5800000C000C000C000C000C00000000000021
:103B68000000803F803F8001000300030006000C36
:103B7800000C0018001800300060807F807F000073
:103B880000000000000F000F000C000C000C000CDF
:103B9800000C000C000C000C000C000C000C000CBD
:103BA800000C000C000F000F00000018001800188F
:103BB800000C000C000C000C0006000600060006B5
:103BC800000300030003000000000000001E001EA8
:103BD80000060006000600060006000600060006AD
:103BE800000600060006000600060006001E001E6D
:103BF8000000000C000C001E00120033003380612E
:103C080080610000000000000000000000000000CB
:103C1800000000000000000000000000000000009C
:103C2800000000000000000000000000000000008C
:103C380000000000E0FF0000000000380018000C41
:103C4800000000000000000000000000000000006C
:103C5800000000000000000000000000000000005C
:103C6800000000000000001F803F80618001801F6D
:103C7800803F80618063807FC038000000000000C2
:103C880000000060006000600060006E007F8073CC
:103C980080618061806180618073007F006E0000B8
:103CA8000000000000000000000000000000001EEE
:103CB800003F807380610060006080618073003F16
:103CC800001E00000000000000008001800180014B
:103CD8008001801D803F8073806180618061806188
:103CE8008073803F801D000000000000000000007D
:103CF800000000000000001E003F00738061807F0C
:103D0800807F00608071003F001E000000000000FE
:103D18000000C007C00F000C000C807F807F000CE3
:103D2800000C000C000C000C000C000C000C000037
:103D3800000000000000000000000000801D803F1F
:103D4800807380618061806180618073803F801DA5
:103D580080018063007F003E00000060006000601A
:103D68000060006F807F8071806180618061806108
:103D78008061806180610000000000000000000692
:103D8800000600000000003E003E00060006000697
:103D980000060006000600060006000000000000FD
:103DA8000006000600000000003E003E0006000677
:103DB800000600060006000600060006000600468B
:103DC800007E003C000000600060006000608061D0
:103DD80000630066006C007C00760063006380610D
:103DE800C0600000000000000000003E003E000629
:103DF800000600060006000600060006000600068B
:103E08000006000600060000000000000000000098
:103E180000000000000080DDC0FFC0CEC0CCC0CCD8
:103E2800C0CCC0CCC0CCC0CCC0CC000000000000CE
:103E380000000000000000000000006F807F80711B
:103E48008061806180618061806180618061000043
:103E58000000000000000000000000000000001E3C
:103E6800003F807380618061806180618073003F62
:103E7800001E00000000000000000000000000001C
:103E8800006E007F807380618061806180618073D3
:103E9800007F006E006000600060006000000000AD
:103EA80000000000801D803F807380618061806118
:103EB80080618073803F801D8001800180018001C6
:103EC800000000000000000000000067803F00398B
:103ED800003000300030003000300030003000008A
:103EE8000000000000000000000000000000001EAC
:103EF800803F80610060007F803F80018061007F9B
:103F0800001E00000000000000000000000800186B
:103F18000018007F007F001800180018001800180B
:103F28000018801F800F0000000000000000000043
:103F38000000000000008061806180618061806114
:103F4800806180618063807F803D00000000000008
:103F580000000000000000000000C06080318031D7
:103F68008031001B001B001B000E000E0006000025
:103F7800000000000000000000000000000080DDDC
:103F880080DD80DD00550055005500770077002260
:103F980000220000000000000000000000000000F7
:103FA8000000806100330033001E000C000C001E6E
:103FB80000330033806100000000000000000000B2
:103FC8000000000080618061803100330033001BF5
:103FD800001B001B000E000E000E001C007C007071
:103FE80000000000000000000000C07FC07F8001CA
:103FF80000030006000C00180030C07FC07F0000DE
:104008000000000080038007000600060006000686
:104018000006000E001C001C000E0006000600062C
:10402800000600068007800300060006000600065A
:104038000006000600060006000600060006000648
:104048000006000600060006000600060038003CD0
:10405800000C000C000C000C000C000E0007000700
:10406800000E000C000C000C000C000C003C00388A
:104078000000000000000000000000000000803880
:10408800807F0047000000000000000000000000E2
:10409800000000000000000000000000010203040E
:1040A80006070809000000000102030402030405D2
:1040B800060708090A0B0C0D0E0F1010010230310B
:1040C8003233343536373839616263646566676818
:1040D800696A6B6C6D6E6F707172737475767778D0
:0440E800797A0000E1
:0440EC003501000892
:0440F00011010008B2
:1040F4000B120000403300080024F40010000000FC
:0441040001000000B6
:0400000508001325B7
:00000001FF
